:100000000203B17DC37DA27EB400177E940012026C
:10001000004C4005E47AC9B0227AC9B00BC422541E
:100020000F2490D43440D430F30CBEB0414007BE0E
:10003000B05B500224204CCC68021BC00B84D389D7
:10004000944CCC680B742012003680F5CA3B6D8846
:100050009F337CAE7EA9B00BA47007C37D38DA3B1A
:100060008994B42569C2F37EA9B00BA4A5F824D065
:10007000BEB00A501B7E500A20F60DAC5CA52D7C4C
:10008000CB70034EF00180DDAC5DA52D7CDB80D50F
:1000900024CFBEB01AA5E850055E00DFD2F390026F
:1000A000B2A3E4936011BCB078F77414934CAB30F6
:1000B000F6B34EF08080AEA3E4936010BCB078F746
:1000C0007413937C3B741D937C2B89147CB0801338
:1000D000742012003620F205BEC00250F31BB50991
:1000E000BB00011200360200411BB50BB8104D11C8
:1000F00078047E14800020F21E4CCC681A7D31E416
:100100007E39804C8868070B3404BCBD78F2C2F697
:10011000CA19120214DA197E19B060CACA1912007B
:1001200036DA190B144CDD68EE1BD078EA80B77E06
:10013000101080037E10085EB05F800AD2F67E1039
:100140000A80057E100AC2F66D119F117E00201BE9
:10015000B47EB97030F6021A3720F1051BB47EB9AF
:100160006030F6041A261A2430F0051BB50BB820AF
:10017000A5EC3382F692F6500A7CEA9F229F217FFB
:10018000127CAE4C44780F7C457C567C676C772E95
:1001900000F878EF80122F117CB3337C3B9CB14088
:1001A000047C3B0B70A5D8EE7CB230E005DAB8C415
:1001B0004C3BCA380B207E00207E3000BE18000069
:1001C00078C1BE1008780730F404C2F480B5CA289C
:1001D0007CB2BCBD38027CBD120214DA28BC2D50A2
:1001E0000A1BD0E4CA2812001F80F07CB213DAB8D0
:1001F0004004C4CAB8C4CA28BEF08040095CDD7897
:1002000005A5DA0260065EF07F12001FDA28A5DA83
:10021000DA020041BEF001680F30F402240220F53A
:100220000620F70330F6010420F229BCBC5025CA91
:10023000B87CBF13B0E67420501174307C8A5E80A5
:10024000F068081202545EA00F8003120036DAB87C
:10025000BCBC78DB30F40F7430120036745830F3C5
:1002600002747812003630F605742D020036742BB5
:1002700020F5F8742020F7F3221BB47EB9B010F1FA
:10028000021BB420F60B30E704F404D2F27CCB80DE
:100290000520E7057CDB0200655EF07F80F81BB57A
:1002A0000BB81030F0076D221B18200B151B18809F
:1002B0000200502D2B204C4248232E0053584F440F
:1002C000494355502A4E000420800102001040E9A5
:1002D0002F343C3CD5432F799E00010101010001E0
:1002E00001020275E900A9D7BA75EA007593007595
:1002F000940075910075920075950075960075B122
:100300000075B20075B30075B40075C90075CA00F8
:1003100075CB0075CC0075E10075E200E47E34FE1B
:10032000B17E24007E7A1BB07E1BB044017A1BB0E4
:10033000E47E34FECC7A1BB074687E14FEC87E0462
:10034000007E7A0BB074017A1BB0E47E34FEB27A80
:100350001BB07E1BB044027A1BB0E47E34FED07A20
:100360001BB074EF7E34FED17A1BB0120388748008
:100370007E34FEDD7E24007E7A1BB074817E34FEE6
:10038000C07A1BB0D2AF80FE74077E34FED27E24CA
:10039000007E7A1BB074CF7E34FED37A1BB0740219
:1003A0007E34FED57A1BB074587E34FED67A1BB0EC
:1003B000227584017E44041FE47A49B01B4478F915
:1003C0007EF800160203C71202E36D337E24800418
:1003D0001200037E3480040203DA7D236D33800231
:0A03E0000B347E29B00B2470F722C5
:00000001FF
